:100000000C9417060C947D290C94AA290C943F0695
:100010000C943F060C943F060C943F060C943F064C
:100020000C943F060C943F060C94C50C0C943F06B0
:100030000C943F060C943F060C943F060C943F062C
:100040000C94D7290C943F060C94912D0C94CC2D34
:100050000C943F060C943F060C943F060C943F060C
:100060000C943F060C943F06A61CAD1CAD1CA61CB0
:10007000AD1CAD1CAD1CAD1CAD1CAD1CAD1CAD1C38
:10008000AD1CAD1CAD1CAD1CAD1C1B1CAD1CAD1CBA
:10009000AD1CAD1CAD1C7E1BAD1CAD1CAD1CAD1C48
:1000A000AD1CAD1CAD1CAD1CAD1CAD1CAD1CAD1C08
:1000B000AD1CAD1CAD1C271C271C271C271C271C96
:1000C000271C271C271C271CAD1CAD1CAD1CAD1C00
:1000D000AD1CAD1C831B261C261C261C261CAD1C1F
:1000E000371C3F1C471C4F1C571C5F1C671C6F1C98
:1000F000791C831C8D1C971CCA1B8A1BAD1CAD1C54
:10010000AD1CAD1C1B1CAD1CAD1CAD1CAD1CAD1C39
:10011000AD1CAD1CAD1C251C251C251C251CAD1CB7
:10012000371C3F1C471C4F1C571C5F1C671C6F1C57
:10013000791C831C8D1C971CCA1B8A1BAD1CAD1C13
:10014000AD1CAD1C1B1CDE1CDE1CDE1CDE1CDE1C04
:10015000DE1CDE1CDE1CDE1CDE1CDE1CDE1CDE1CCF
:10016000FE1DFE1DFE1DFE1DFE1DFE1D251D2F1D5F
:10017000391D431DA91DB31DC11DD21D6F1EDF1EDC
:10018000B01EB51EBA1EBF1EC41EC91ECE1EDF1E67
:10019000D91EF9250E261A262326302656265E2637
:1001A00081266E26456E746572206D656E752E2EE5
:1001B0002E00546F67676C6564206D6963726F50C1
:1001C000504D00546F67676C656420696E76657288
:1001D0007465642050504D2100546F67676C6564EE
:1001E000205458206D7574696E672100546F6767DD
:1001F0006C65642074656C656D657472792100505E
:10020000726F746F636F6C206572726F72207769A2
:1002100074682052580054696D656F757420776852
:10022000656E20636F6E6E656374696E6720746FB0
:1002300020525800507265737320616E79206B658F
:100240007920746F2063616E63656C00436F6E6E1E
:10025000656374696E6720746F2052582C20706F2C
:100260007765722075702074686520525820287751
:100270006974682062696E6420706C7567206966B5
:10028000206E6F74207573696E6720616C77617979
:10029000732062696E642900546F67676C6564201F
:1002A00027696D6D656469617465206F757470751B
:1002B000742700546F67676C65642027736C6176E0
:1002C00065206D6F64652700546F67676C656420F7
:1002D00027616C776179732062696E642700546FBF
:1002E00067676C65642050504D206368616E6E6571
:1002F0006C206C696D6974005365742052535349C6
:1003000020696E6A656374696F6E206368616E6EE2
:10031000656C2028303D3D64697361626C6529001D
:100320005365742050504D206D696E696D756D2058
:1003300073796E630053657420626561636F6E202C
:10034000696E74657276616C0053657420626561D4
:10035000636F6E2064656C6179005365742062651B
:1003600061636F6E206672657175656E6379206971
:100370006E20487A3A20303D64697361626C652C66
:100380002050783D504D52206368616E6E656C2040
:10039000782C2046783D465253206368616E6E6526
:1003A0006C2078005365742050574D2073746F7023
:1003B0002064656C61792028302064697361626C07
:1003C00065642C20312D323535203D3D20302E31D5
:1003D00073202D2035306D696E29005365742050CF
:1003E000504D2073746F702064656C6179202830E3
:1003F0002064697361626C65642C20312D3235355F
:10040000203D3D20302E3173202D2035306D696E1A
:100410002900536574206661696C736166652064A8
:10042000656C61792028302064697361626C656451
:100430002C20312D323535203D3D20302E3173209A
:100440002D2035306D696E29002A2A2A2A2A2A2A67
:100450002A2A2A2A2A2A2A2A2A2A2A2A2A2A2A2AFC
:100460002A2A2A2A2A2A0052582041636B656420CE
:100470002D2072657665727420737563636573737E
:1004800066756C21002A2A2A2A2A2A2A2A2A2A2A36
:100490002A2A2A2A2A2A2A2A2A2A2A2A2A2A2A2ABC
:1004A0002A2A002A2A2A2A2A2A2A2A2A2A2A2A2AD6
:1004B0002A2A2A2A2A2A2A2A2A2A2A2A2A2A2A2A9C
:1004C0000052582041636B6564202D207570646173
:1004D0007465207375636365737366756C21002A98
:1004E0002A2A2A2A2A2A2A2A2A2A2A2A2A2A2A2A6C
:1004F0002A2A2A2A2A2A2A2A2A2A2A2A0056616CE1
:1005000069642063686F69636573206172653A206E
:100510005B315D2D5B31365D20286368616E6E65F1
:100520006C20312D31362900536574206F7574703D
:10053000757420666F7220706F727420005B585D56
:100540002061626F7274206368616E6765732061F9
:100550006E64206578697420525820636F6E6669F6
:1005600067005B535D207361766520736574746901
:100570006E677320746F205258005B525D20726565
:10058000766572742052582073657474696E67734F
:1005900020746F2064656661756C747300557365B3
:1005A000206E756D62657273205B312D445D207421
:1005B0006F206564697420706F727473205B452DC1
:1005C000515D20666F722073657474696E67730085
:1005D000202D20726563656976657220636F6E6693
:1005E0006967757261746F722C207278207377203E
:1005F000000A0A6F70656E4C52536E672000536597
:10060000742073657269616C2062617564726174D3
:10061000653A200056616C69642063686F696365A0
:10062000733A2031202D20342B34202F2032202DDE
:100630002038202F2033202D20382B34202F203419
:10064000202D203132202F2035202D2031322B3407
:10065000202F2036202D203136005365742043682A
:10066000616E6E656C20636F6E6669673A20005339
:1006700065742044617461726174652028302D3284
:10068000293A200053657420486F70206368616EBA
:100690006E656C7320286D61782032342C20736570
:1006A0007061726174656420627920636F6D6D6141
:1006B00073292076616C69642076616C756573209E
:1006C000312D3235353A2000536574206368616EF0
:1006D0006E656C2073706163696E672028783130B5
:1006E0006B487A293A200053657420524620706F77
:1006F0007765722028302D37293A20005365742001
:100700005246206D616769632028686578292065F5
:100710002E672E20307844454144463030443A20FC
:10072000005365742062617365206672657175653A
:100730006E63792028696E20487A293A20005B5A36
:100740005D20656E74657220726563656976657299
:1007500020636F6E66696775726174696F6E20756C
:1007600074696C79005B465D20646973706C6179B3
:100770002061637475616C206672657175656E6366
:100780006965732075736564005B525D2063616CFD
:1007900063756C6174652072616E646F6D206B654A
:1007A0007920616E6420686F70206C697374005BDF
:1007B000495D207265696E697469616C697A65204A
:1007C00073657474696E677320746F20736B6574DE
:1007D00063682064656661756C7473005B585D20A6
:1007E000726576657274206368616E6765732061F7
:1007F0006E642065786974206D656E75005B535D6D
:1008000020736176652073657474696E67732074F4
:100810006F20454550524F4D20616E6420657869C8
:1008200074206D656E7500557365206E756D62651B
:100830007273205B302D395D20746F20656469749C
:1008400020706172616D657465727300202D205394
:10085000797374656D20636F6E6669677572617414
:10086000696F6E000A0A6F70656E4C52536E672096
:10087000005129204F7574707574206265666F721F
:1008800065206C696E6B20283D465329203A200074
:10089000502920536C617665206D6F646520286552
:1008A00078706572696D656E74616C293A20004FCD
:1008B000292054696D65642042494E4420617420AA
:1008C0007374617274757020203A20004E29205094
:1008D000504D206F7574707574206C696D69746506
:1008E0006420202020203A200044495341424C45B6
:1008F00044004D292050504D205253534920746FCD
:10090000206368616E6E656C202020203A20004CC8
:10091000292050504D206D696E696D756D20737979
:100920006E63202875732920203A200044495341E2
:10093000424C4544004B29204661696C73616665F1
:1009400020626561636F6E20696E74762E20283197
:100950002D32353573293A20004A29204661696CC9
:100960007361666520626561636F6E2064656C61AA
:10097000792028302D323535203D3E20313073200E
:100980002D203135306D696E293A200049292046E5
:1009900061696C7361666520626561636F6E206674
:1009A00072712E203A200048292050574D20737430
:1009B0006F702064656C6179202020202020203A0F
:1009C000200047292050504D2073746F70206465BB
:1009D0006C6179202020202020203A200046292008
:1009E0004661696C736166652064656C617920207D
:1009F00020202020203A200050574D206368616E4F
:100A00006E656C200066756E6374696F6E3A2000C7
:100A10002920706F72742000506F776572546F7761
:100A2000657200445446205548462033322D626991
:100A3000742031306368004F70656E4C52536E679E
:100A40005258206D696E6920342F36636800466CF9
:100A50007974726F6E2F4F72616E676552582055B0
:100A600048462038636800525820747970653A20EF
:100A70000044697361626C656400487A00203D3D02
:100A8000200043616C63756C617465642070616300
:100A90006B657420696E74657276616C3A200042F1
:100AA00029204D6963726F202868616C6629205087
:100AB000504D202020203A00412920496E76657251
:100AC0007465642050504D20696E20202020203A0B
:100AD000003029204D7574652062757A7A65722020
:100AE000286D6F73746C79293A0039292053657227
:100AF00069616C2062617564726174653A00736D3E
:100B0000617274506F7274004672536B7900547244
:100B1000616E73706172656E740044697361626CBA
:100B200065640038292054656C656D657472793A86
:100B300020202020202020003729204368616E6E6D
:100B4000656C20636F6E6669673A20200036292045
:100B500044617461726174652028302D32293A2015
:100B6000202000352920486F70206368616E6E6513
:100B70006C733A2020202020003429204368616EC5
:100B80006E656C2073706163696E673A2020003374
:100B90002920524620706F7765722028302D372922
:100BA0003A202020003229205246206D6167696377
:100BB0003A202020202020202020003129204261BE
:100BC0007365206672657175656E63793A202020C1
:100BD0000000000000240027002A0000000000257B
:100BE0000028002B0000000000230026002900043C
:100BF00004040404040404020202020202030303C4
:100C000003030301020408102040800102040810BD
:100C1000200102040810200000000700020100006B
:100C2000030406000000000000000000742F1124DF
:100C30001FBECFEFD8E0DEBFCDBF13E0A0E0B1E034
:100C4000EAE2F1E602C005900D92A839B107D9F7A2
:100C500016E0A8E9B3E001C01D92AD35B107E1F798
:100C60001CE0CEE2DCE004C02297FE010E9470305E
:100C7000CC32D107C9F70E94B92F0C9493300C9451
:100C80000000A0E0B0E0E7E4F6E00C943F30EC01B7
:100C9000A880B980CA80DB80A114B104C104D1044A
:100CA00041F484E2A82E89EDB82E8BE5C82E87E0AA
:100CB000D82EC601B5012DE133EF41E050E00E948E
:100CC0001C3027EA31E440E050E00E94C82F7B014D
:100CD0008C01C601B5012DE133EF41E050E00E94E7
:100CE0001C30CA01B9012CEE34EF4FEF5FEF0E94C8
:100CF000C82F6E0D7F1D801F911F97FF04C061508C
:100D0000704080409048688379838A839B839B01ED
:100D1000AC015F77B901CA01CDB7DEB7EAE00C9448
:100D20005B300E944106089581EB92E00E944106EB
:100D300008956093B1027093B2028093B3029093CE
:100D4000B4020895A0E0B0E0E8EAF6E00C94383090
:100D5000EC012B016A016115710519F0FB0191830A
:100D60008083C114D10449F0C6010297839728F00B
:100D700020E030E040E050E0DCC0A9908A2D90E017
:100D80000E948830892BC9F7FDE2AF1621F4A990A3
:100D90003324339405C08BE2A81609F4A9903324B8
:100DA000C114D10421F0E0E1CE16D10411F5F0E335
:100DB000AF1669F48881883711F0883541F4A9802D
:100DC000229682E0382A20E1C22ED12C12C0C11412
:100DD000D10479F4E0E3AE1659F199E9E92E99E9E5
:100DE000F92E99E9092F99E1192F8AE0C82ED12C03
:100DF0003AC0FAE0CF16D10491F080E1C816D104D0
:100E000029F0E8E0CE16D104F9F415C0BFEFEB2EBF
:100E1000BFEFFB2EBFEF0B2FBFE01B2F24C0A9E9B4
:100E2000EA2EA9E9FA2EA9E90A2FA9E11A2F1BC077
:100E3000F8E0CF2ED12CEFEFEE2EEFEFFE2EEFEFFE
:100E40000E2FEFE11E2F0FC09601442737FD40956E
:100E5000542F6FEF7FEF8FEF9FEF0E94FA2FC901A2
:100E6000DA017C018D0120E030E040E050E060E0FC
:100E70003601882477FC8094982C70EDB72EBA0C3C
:100E8000F9E0FB1570F48A2D81548A3118F499EC3D
:100E9000B92E06C08A2D81568A3148F589EAB82EC6
:100EA000BA0C8B2D90E08C159D050CF56F3FE9F089
:100EB000E216F30604071507B8F0CA01B901A40148
:100EC00093010E94C82F9B01AC018B2D90E0A0E004
:100ED000B0E0280F391F4A1F5B1F281739074A0740
:100EE0005B0710F061E001C06FEFA990C6CF41141D
:100EF000510451F0662311F0219703C031FE04C064
:100F00002297F201D183C08330FE07C050954095EF
:100F1000309521953F4F4F4F5F4F67FF0AC082E2E8
:100F200090E090935C0680935B062FEF3FEF4FEFCE
:100F30005FEFB901CA01CDB7DEB7E1E10C945430DF
:100F4000FC0188279927E89421912032E9F3293080
:100F500010F02E30C8F32B3241F02D3239F4689462
:100F600004C00E94F507820F911D219120532A3061
:100F7000C0F31EF4909581959F4F089548E953E082
:100F80000E94C3070895009731F4DA018D919C9176
:100F9000009709F40EC0DC01FB013D912191222351
:100FA00019F03217C9F3FACF332331F4DA011D9265
:100FB0001C928827992708951197AF93BF93FB013F
:100FC0003D912191321771F4332321F48827992719
:100FD000119702C01E921196FA01A193B0839F91BE
:100FE0008F910895222369F7EACF7AE0979F902D99
:100FF000879F802D910D1124089580919A0381304F
:1010000019F482E080939A0380919A03833019F453
:1010100084E080939A030895E3E0F0E089E0809310
:101020005700849190E08670863009F491E0892F12
:1010300008951F93182F0E940C08882379F09FB7FA
:1010400081E08093A305F894A89588E180936000DF
:1010500010936000112309F0A8959FBF1F91089578
:10106000382F20E08091350590913605822793270F
:1010700040E061E270E19C01220F331F97FF04C042
:10108000C9018627972701C0C9014F5F483099F7EA
:101090009093360580933505089587E38093D003B8
:1010A00080E092ECA1E0B0E08093D1039093D20372
:1010B000A093D303B093D40387E08093DD0380EC47
:1010C0009AECA9E8B6E38093D5039093D603A09356
:1010D000D703B093D80385E08093DE038DEE9EEFB7
:1010E000ADEABEED8093D9039093DA03A093DB03BE
:1010F000B093DC03AFEDB3E080E090E0863010F019
:10110000E0E004C0FC01EF57FC4FE081ED93019655
:101110008831910599F782E08093F7038AE0809304
:10112000F803089580EC97EFAAEBB7E380939D0353
:1011300090939E03A0939F03B093A00380E090E060
:10114000A0E0B0E58093A1039093A203A093A30332
:10115000B093A403E5EAF3E080E081938F5F8031F0
:10116000E1F708958436910520F4BC0180E090E019
:1011700025C08E3B910550F48A559040BC0180E01B
:1011800090E02AE030E040E050E016C0823D91055A
:1011900050F4845B9040BC0180E090E024E630E0B5
:1011A00040E050E009C08D5C9040BC0180E090E0E0
:1011B00028E532E040E050E00E94C82F24E630E00D
:1011C00040E050E00E94C82F089590E08C599F4F56
:1011D0000E94B2080895DC019896EC91F0E0E77067
:1011E000F070E758FC4F808108958F929F92AF92E4
:1011F000BF92CF92DF92EF92FF920F931F938C01D9
:101200000E94EB08D80197962C9130E043E150E022
:10121000249FF001259FF00D349FF00D1124EB5415
:10122000FD4F80809180A280B38090E00F96AA2726
:1012300097FDA095BA2FBC01CD0120E43FE14DE719
:1012400050E00E94C82FA50194010E94FA2F690165
:101250007A0180ED97E0A0E0B0E0C80ED91EEA1E4A
:10126000FB1ED80198968C91887181F060E07EEE2B
:101270008AEB9BE0A50194010E94FA2F28513C4F74
:101280004F4F5F4FC20ED31EE41EF51E87EE93E054
:10129000A0E0B0E0C80ED91EEA1EFB1EC701B601D1
:1012A00028EE33E040E050E00E94FA2FCA01B90175
:1012B00028EE33E040E050E00E94C82F1F910F91CC
:1012C000FF90EF90DF90CF90BF90AF909F908F9066
:1012D00008958F3F910509F010F480E0089522E011
:1012E0008030920710F481E008958050934010F010
:1012F00083E0089582E00895CF92DF92FF920F93EA
:101300001F93CF93DF93F82FEB016A01182F1695E7
:10131000E0E088819981D6018C938A819B81119626
:101320008C9311978C819D8112968C9312978E814C
:101330009F8113968C931397288139814A815B8111
:101340006C817D818E819F819295990F990F907C00
:10135000832F8370982B852F8370880F880F982B8D
:10136000872F83708295807F982B14969C9385E0BD
:1013700090E0C80ED91E2896EF5F1E1750F6F0FFBA
:1013800021C0888199810E946909F82E8A819B81F8
:101390000E946909182F8C819D810E946909082F7C
:1013A0008E819F810E946909F294FF0CFF0C70EC02
:1013B000F7221295107F1F29182B000F000F012B09
:1013C000D6010C93DF91CF911F910F91FF90DF9089
:1013D000CF90089523E08032920718F420E030E0A7
:1013E00026C023E0883E920748F49C012F513340E9
:1013F00054E0369527955A95E1F719C027E0803DCE
:10140000920720F49C012C5D334011C028E08839FC
:10141000920718F02FEF33E00AC09C01285C374098
:1014200044E0369527954A95E1F72D503C4FC90188
:1014300008958C30910548F49C0174E0220F331F0D
:101440007A95E1F7285D3C4F17C023E0843F92076F
:1014500020F49C0124523C4F0FC024E080309207BE
:1014600018F020E938E008C09C012657334F64E0AB
:10147000220F331F6A95E1F7C90108959C01369543
:10148000279525753575821B930B9C0136952795FD
:10149000369527952373337383739373280F391FFE
:1014A000C901E4E096958795EA95E1F7820F931FCD
:1014B0008F709F7021E031E0AC01429FC001439FDB
:1014C000900D529F900D1124892F0895882339F093
:1014D0002D9800002B9A00002D9A000008952D9859
:1014E00000002B9800002D9A000008952D9A00000E
:1014F00083B12D98000090E0B4E096958795BA9559
:10150000E1F7817008950F931F93082F5C9A2D982F
:101510005C9810E0802F80780E94660A000F1F5FA1
:101520001830C1F72D981F910F9108958F770E9461
:10153000830A08950F931F93082F10E0802F80785F
:101540000E94660A000F1F5F1830C1F72D981F9187
:101550000F9108950F931F932D9880E000E0182FAE
:10156000110F0E94760A810F0F5F0830C1F71F919B
:101570000F9108950E94960A0E94AA0A5C9A089503
:101580001F93162F80680E94830A812F0E949A0A57
:101590005C9A1F9108951F931091D9031827E0EDCD
:1015A000F3E0E80FF11D89E767850E94C00A8DE32B
:1015B000612F0E94C00A82E4612F0E94C00A1F911D
:1015C000089586E20E94BA0A08950F931F938C0132
:1015D0008CE1F80164810E94C00A8DE1F801658107
:1015E0000E94C00A8EE1F80166810E94C00A80E272
:1015F000F80167810E94C00A81E2F80160850E94BB
:10160000C00A82E2F80161850E94C00A83E2F80103
:1016100062850E94C00A84E2F80163850E94C00AC4
:1016200085E2F80164850E94C00A8AE2F8016585B6
:101630000E94C00A8EE6F80166850E94C00A8FE605
:10164000F80167850E94C00A80E7F80160890E945E
:10165000C00A81E7F80161890E94C00A82E7F801A7
:1016600062890E94C00A1F910F910895EF92FF9224
:101670000F931F93CF93DF937B018C01603028E39E
:1016800072072CE982072CE1920728F520E836E959
:1016900048E950E00E94FA2FE9016897B90180E01B
:1016A00090E020E839E647E65FEF0E94C82F6E0D14
:1016B0007F1D801F911F32E0660F771F881F991FC3
:1016C0003A95D1F721E732E040E050E00E94FA2F4E
:1016D000890180E421C020E03DE241E351E00E9425
:1016E000FA2FE9016897B90180E090E020E033ED3E
:1016F0004EEC5EEF0E94C82F6E0D7F1D801F911F64
:10170000660F771F881F991F21E732E040E050E005
:101710000E94FA2F890180E69E012F71622F680FC7
:1017200085E70E94C00A86E7612F0E94C00A87E70A
:10173000602F0E94C00ACDB7DEB7E6E00C945F30A0
:10174000682F8DE60E94C00A08959F92AF92BF92C3
:10175000CF92DF920F93DF93CF9300D000D0CDB71D
:10176000DEB7982E83E00E94BA0A8093F90384E0E2
:101770000E94BA0A8093FA0386E060E00E94C00AE1
:1017800087E061E00E94C00A89E06FE70E94C00A1A
:101790008AE065E00E94C00A8BE062E10E94C00A14
:1017A0008CE065E10E94C00A8DE06DEF0E94C00AE6
:1017B0008EE060E00E94C00A992019F084E193E075
:1017C00008C08091F70323E1829FC00111248B544C
:1017D0009D4F0E94E50A80E36CE80E94C00A82E304
:1017E0006FE00E94C00A83E362E40E94C00A84E3BF
:1017F0006AE00E94C00A85E36AE20E94C00A86E3AA
:101800006DE20E94C00A87E364ED0E94C00A88E38B
:1018100060E00E94C00A89E360E00E94C00A99204B
:1018200049F065E8A62E61ECB62E61ECC62E6EED91
:10183000D62E08C0A090D903B090DA03C090DB0385
:10184000D090DC030AE38D2D9927AA27BB27898333
:101850009A83AB83BC83802F69810E94C00A802F4A
:101860008B5F69810E94C00ADC2CCB2CBA2CAA2485
:101870000F5F0E3341F783E46FEF0E94C00A84E4E8
:101880006FEF0E94C00A85E46FEF0E94C00A86E4F1
:101890006FEF0E94C00A992019F08DE666E003C040
:1018A0008DE66091DD030E94C00A89E760E00E9436
:1018B000C00A8AE76091DE030E94C00A83E760E005
:1018C0000E94C00A84E760E00E94C00A992029F0C3
:1018D00060EC7AEC89E896E308C06091D5037091DA
:1018E000D6038091D7039091D8030E94360B0F90B6
:1018F0000F900F900F90CF91DF910F91DF90CF90CD
:10190000BF90AF909F90089587E061E00E94C00A69
:101910008EE764E20E94C00A88E063E00E94C00A89
:1019200088E060E00E94C00A87E065E00E94C00A8B
:1019300085E062E00E94C00A83E00E94BA0A8093B8
:10194000F90384E00E94BA0A8093FA030895582F9D
:1019500040919E04842F90E0FC01EF70F0709F0195
:101960002F5F3F4F74E0959587957A95E1F728179B
:10197000390751F0E257FB4F5083842F8F5F8F70F0
:10198000407F842B80939E0408951F920F920FB680
:101990000F9211241F932F933F934F935F936F9355
:1019A0007F938F939F93AF93BF93CF93DF93EF93E7
:1019B000FF93C0918600D09187002091E20430917E
:1019C000E3048091C104882309F062C0BE01621B58
:1019D000730B2091A1033091A2034091A303509176
:1019E000A40325FD02C07695679589E0653C7807DC
:1019F000B8F1809147031CE1569547953795279597
:101A00001A95D1F7211531054105510521F421E041
:101A100030E040E050E090E0A0E0B0E02817390767
:101A20004A075B07D0F4809147038F3FB1F020E075
:101A30000EC0E22FF0E0EE0FFF1FDF01AE53BB4FF1
:101A40008D919C91E95DFC4F918380832F5F809104
:101A50004703281770F31092C0041092470318C070
:101A600082E06D3B780760F180914703803140F55B
:101A700010914703CB010E94EA09E12FF0E0EE0F3D
:101A8000FF1FEE53FB4F918380831F5F109347032B
:101A9000D093E304C093E204FF91EF91DF91CF91E3
:101AA000BF91AF919F918F917F916F915F914F9176
:101AB0003F912F911F910F900FBE0F901F9018957F
:101AC0008FEF80934703E4CF83E0809380008AE91F
:101AD000809381008091A10386FD05C080918100E3
:101AE0008064809381008FEF9FEF909389008093B3
:101AF000880080916F00806280936F0008956F303E
:101B000018F086958058089589E0689F802D1124EB
:101B10000895882319F460E071E002C063E071E089
:101B200089E396E00E947C2D0895A0E0B0E0EBE907
:101B3000FDE00C944130182F0E942D2A9B01AC012E
:101B400080912F0590913005A0913105B09132051B
:101B500069017A01C81AD90AEA0AFB0AD701C60143
:101B600089589341A040B04010F010922E05209368
:101B70002F05309330054093310550933205209165
:101B8000C104822F81508230E8F580912E05882390
:101B900009F44FC1813011F482E0BCC1803108F0FA
:101BA00035C1E82FF0E0EE53FB4F10838F5F809339
:101BB0002E05803109F0B0C1A4ECB4E0213039F435
:101BC0001196EC911197E695E6958C9109C08D914F
:101BD0009C911197E92FE695E695E6959695879560
:101BE000E03140F4F0E090E0EE0FFF1FE95DFC4FC4
:101BF000918380831092C004129684E0A23DB807BE
:101C0000E9F68AC1233009F004C180912E058823AA
:101C100021F41F3009F080C10CC1883130F4E82F65
:101C2000F0E0EF53FB4F108374C1883109F0EEC030
:101C3000112309F0EBC0C0E0D0E00BE010E0DE01C2
:101C400063E0AA0FBB1F6A95E1F7C09FB001C19F77
:101C5000700DD09F700D1124FB01EE53FB4F80815E
:101C60002181922F977095958795FD01EE0FFF1FAB
:101C7000E95DFC4F91838083FB01ED53FB4F308185
:101C80003695369536952181422F4295440F407EF8
:101C9000842F832B269526952695922F97709595C0
:101CA0008795FD01EE0FFF1FE75DFC4F9183808359
:101CB000FB01EC53FB4F808182958695869583705E
:101CC0004181942F990F990F292F282B42954695E2
:101CD0004695437082818170880F880F382F342B8E
:101CE00035952795FD01EE0FFF1FE55DFC4F318314
:101CF0002083FB01EA53FB4F308136952181422F2F
:101D0000479544274795842F832B2695922F9770CC
:101D100095958795FD01EE0FFF1FE35DFC4F9183C5
:101D20008083FB01E953FB4F308132953F70218165
:101D3000422F4295407F842F832B22952F70922F24
:101D4000977095958795FD01EE0FFF1FE15DFC4FA4
:101D500091838083FB01E853FB4F8081881F882794
:101D6000881F4181942F990F292F282B441F442726
:101D7000441F82818370880F382F342B3595279527
:101D8000FD01EE0FFF1FEF5CFC4F31832083FB0151
:101D9000E653FB4F3081369536952181422F42958F
:101DA000440F440F407C842F832B26952695922F39
:101DB000977095958795AA0FBB1FFD01ED5CFC4FB1
:101DC0009183808365537B4FFB012081229526956B
:101DD00027704181342F330F330F330F832F822B22
:101DE000942F92959695977095958795AB5CBC4F7F
:101DF00011969C938E932196C230D10509F01FCF86
:101E00008091D80483FD02C01092C00410922E0568
:101E100083C0243009F080C040912E05442359F43A
:101E2000183AB1F4109236051092350588EA0E94EE
:101E3000300881E06FC0413019F41093330504C0BD
:101E4000423031F410933405812F0E9430085DC078
:101E500060913405262F30E0220F331FE42FF0E08D
:101E6000C90102968E179F0734F0433268F7E15498
:101E7000FB4F1083E9CF2D5F3F4F409135055091C7
:101E80003605E217F30749F4912F80E048275927D8
:101E9000509336054093350538C0812F90E04817A0
:101EA000590789F580913305813069F5613118F062
:101EB00080E180933405D090340542ECE42E44E078
:101EC000F42E00E010E01BC0F701D081C0E081815A
:101ED00090E08C2B9D2B33E0969587953A95E1F712
:101EE0000E94EA09F801EE0FFF1FE95DFC4F9183A4
:101EF00080830F5F1F4F82E090E0E80EF91E0D1502
:101F000018F31092C00410922E0580912E0588239C
:101F100019F08F5F80932E05CDB7DEB7E8E00C9403
:101F20005D30FF920F931F93CF93DF93182F092FEC
:101F3000F62E8EE30E94C00A212F302FC901EC013A
:101F400010E005C08FE769910E94C00A1F5F1F154E
:101F5000C8F385E064E00E94C00A83E00E94BA0AE8
:101F60008093F90384E00E94BA0A8093FA030E94E6
:101F70002D2A6093FB037093FC038093FD039093E1
:101F8000FE0387E069E00E94C00A81E080939A0323
:101F9000CDB7DEB7E5E00C9460300E94910F8091E0
:101FA0009A038130D9F40E942D2A2091FB033091AD
:101FB000FC034091FD035091FE03621B730B840BE5
:101FC000950B605A76488140904040F4E8CF89E311
:101FD00096E067E071E00E947C2D089580919A035D
:101FE0008130A9F3089589E396E06EE70E94342FCB
:101FF0000895A0E0B0E0EFEFFFE00C9440306C01FA
:1020000089E396E06EE70E94342F760100E010E04D
:10201000C0E0D0E0B0E2BB2E0AC00830110521F4C8
:102020009E012095F60120870894E11CF11CF70120
:102030006081862F8D57823040F489E396E06DE70A
:102040000E94342FF70160816B2589E396E00E949E
:10205000342F0115110551F0F70180819E01280FE1
:10206000311DC32FDD27C20FD31FD0700F5F1F4F4D
:102070000930110591F6CDB7DEB7E9E00C945C307C
:10208000A9E0B0E0E6E4F0E10C944730382FE62F09
:102090008091A30490E0019664E270E00E94E72F33
:1020A000982F8093A30488E9898380E18A83913003
:1020B00071F0913028F0923099F09330E1F416C02D
:1020C00085E08B8381EF8C832F5F2D8317C09B83EB
:1020D00081EF8C8384E6489FC00111249D830EC04C
:1020E00084E08B8381EF8C833D8308C09B8381EFE9
:1020F0008C83ED8303C00E94F30F04C0CE010196D0
:102100000E94F90F2996E2E00C9463300F931F931D
:10211000CF93DF93182F092F89E396E06EE70E9493
:10212000342F212F302FC901EC0110E000E288810B
:102130008D57823040F489E396E06DE70E94342F9A
:1021400088818027888389E396E069910E94342FF3
:102150001F5F193061F789E396E06EE70E94342F24
:10216000DF91CF911F910F910895A9E0B0E0EBEBC3
:10217000F0E10C944730382F8091A304882379F440
:102180008EEF89833A836B83842F90E095958795B2
:102190008C832D83198618861F821E822FC0409142
:1021A0009E04842F90E09C012F70307054E0959530
:1021B00087955A95E1F78217930721F18DEF89836F
:1021C0001A821B82DE01149620E008C0E257FB4F02
:1021D00080818D93405F2F5F263069F0842F90E0DF
:1021E000FC0134E0F595E7953A95E1F78F70907032
:1021F000E817F90759F740939E042A83CE01019608
:102200000E9486108091A30490E0019666E070E041
:102210000E94E72F8093A3042996E2E00C94633098
:102220009F92AF92BF92CF92DF92EF92FF920F9365
:102230001F93B82EA62ED42EC22E902E0E942D2A89
:102240007B018C0180918D0420919F043091A0042A
:102250004091A1045091A2048823B1F0D801C70194
:10226000821B930BA40BB50B815E9E42A040B04035
:1022700020F12C2DDC1408F42D2D8B2D6A2D422FEE
:10228000292D0E94401011C0D801C701821B930B59
:10229000A40BB50B81539547A040B04070F08B2D37
:1022A0006A2D4D2D2C2D0E94B510E0929F04F092C6
:1022B000A0040093A1041093A2041F910F91FF901A
:1022C000EF90DF90CF90BF90AF909F90089589E3FB
:1022D00096E0609100040E94342F08951F93182FF8
:1022E00089E396E0612F0E94342F809100048127BA
:1022F000809300041F9108951F93192F0E946E115F
:10230000812F0E946E111F910895DF92EF92FF922C
:102310000F931F93D82E7B011092000409E316E05F
:10232000C80165EB0E94342FC80162E60E94342F79
:102330008D2D0E946E11C7010E947C111F910F917B
:10234000FF90EF90DF900895E82FF0E0E456FC4F07
:10235000E185E03158F4F894F0E0EE0FFF1FE95DFD
:10236000FC4F0190F081E02D78940DC0E03129F010
:10237000E13129F0E0E0F2E006C082E101C083E152
:102380000E94812BFC01CF0108958CE060E00E9447
:10239000B22A8BE061E00E94B22A8DE061E00E94E7
:1023A000B22A82E060E00E94B22A84E061E00E94EA
:1023B000B22A0895EF92FF920F931F93009771F145
:1023C0009C0140E050E068E478EE81E090E00E94FB
:1023D0001C30C901DA017C018D0183E161E00E94BA
:1023E0001E2B8FEFE816F1040105110539F030F0CE
:1023F000FFEFEF2EF12C012D112D0AC0E114F10495
:102400000105110529F4E1E0EE2EF12C012D112D2D
:10241000E092B3008091B000806107C083E160E08A
:102420000E941E2B8091B0008F7E8093B0001F9180
:102430000F91FF90EF900895A0E2B0E0E2E2F2E1A8
:102440000C943F308CE00E94BA0A882389F589E316
:1024500096E063E171E00E947C2D5E9A409A80E0F4
:102460000E94A50B0E94840C5E98409821C089E3CD
:1024700096E00E94FB2E482F8091C104882321F012
:10248000842F0E94950D14C080912C05E82FF0E058
:1024900031969F012F713070319780912B0590E01C
:1024A0002817390729F0EE5FFA4F408320932C0557
:1024B00089E396E00E94C12E892BC9F680919A0388
:1024C000843009F08EC00E942D2A6093B00470936E
:1024D000B1048093B2049093B30461157105810532
:1024E000910561F481E090E0A0E0B0E08093B00459
:1024F0009093B104A093B204B093B3048091BC0450
:102500009091BD0481609093BD048093BC0483E0EE
:1025100080939A038FE70E94960A09EF14E00E94C5
:10252000AA0AF80181938F01F5E002301F07B9F77D
:102530004091E4048091F904282F30E0842F90E04A
:102540008227932786FF40C080E448274093E40415
:10255000C90188739070C89709F510E014C01F5F17
:102560008091F803E12FF0E084FF06C0E750FB4FB5
:1025700080810E94A70C07C0E750FB4F89E396E0DB
:1025800060810E94342F212F30E08091F90490E087
:10259000877090708217930714F716C02F733070EE
:1025A000232B91F48091FA048093B4048091FB046E
:1025B0008093B6048091FC048093B7048091FF045B
:1025C0008093BE041092BF0480912D05813019F4D0
:1025D00082E080932D0580912D05833011F41092B7
:1025E0002D050E942D2A5B016C018091B804909109
:1025F000B904A091BA04B091BB040097A105B1053C
:10260000C9F086017501E81AF90A0A0B1B0BD801FB
:10261000C701885B9B40A040B04060F00E94E10A87
:102620008093B5041092B8041092B9041092BA04C1
:102630001092BB0480ED93E00E94F5082091AC0459
:102640003091AD044091AE045091AF048601750104
:10265000E21AF30A040B150BE616F706080719072A
:1026600008F428C1A092AC04B092AD04C092AE04AC
:10267000D092AF04A8958091C0048830A0F08091DA
:10268000A1039091A203A091A303B091A4032CE114
:10269000B695A795979587952A95D1F70097A105A7
:1026A000B10509F0A7C18091C0048F5F8093C00479
:1026B000E090B004F090B1040091B2041091B30422
:1026C000E114F1040105110511F180ED93E00E9480
:1026D000F508AE18BF08C00AD10A6A157B058C053B
:1026E0009D0588F48091A10384FD04C080ED97E0EE
:1026F0000E94DA111092B0041092B1041092B20448
:102700001092B30404C080E090E00E94DA1190912E
:10271000E404907C9093E40400912C0510912B0527
:102720000117B1F180912D05823091F59058909369
:10273000E40480ED93E00E94EB08893010F048E05B
:1027400002C0482F415030E013C03F5FA32FB0E0DC
:10275000812F90E0FC01EE5FFA4F2081FD01EC51EA
:10276000FB4F2083AE5DBA4F2C930196182F1F713B
:10277000341710F4101749F710932B05832F895C39
:102780009091E404892B8093E404309322051AC0CD
:1027900020912D052430D1F490912205E3E2F5E05B
:1027A000A5EEB4E0292F30E02E0F3F1F02C081912B
:1027B0008D93E217F307D9F7995C8091E404982B85
:1027C0009093E40483E080932D0538C08091A704A2
:1027D000823061F491609093E4045E9A409A05EA35
:1027E00013E07E010894E11CF11C11C09093E404F5
:1027F0005E984098222319F481E080932D05809102
:102800002D05833061F784E080932D05E8CFF80132
:1028100081918F010E94A411F701819391937F010F
:10282000F3E0053B1F0799F78091F8038770BE011D
:102830006F5F7F4F45EE54E00E947C095D9A419A9C
:102840002091A5042223A1F09091DD03992381F02A
:102850008091A6048F5F8093A6048150821729F48B
:102860001092A604892F815001C0892F0E94A00BCD
:102870008091A4040E94CB0A80ED93E00E94EB08B3
:10288000682F84EE94E00E94910FE091A404EF5F22
:10289000E093A404E83131F0F0E0E053FC4F878589
:1028A000882341F41092A40405C05E9A409A89E0FE
:1028B0008093C0048091F803887171F180919A032C
:1028C000823051F58091BC049091BD04880F991F0E
:1028D0009093BD048093BC0483E080939A030E948C
:1028E000840C0E942D2A6093B8047093B9048093DD
:1028F000BA049093BB04611571058105910561F4DB
:1029000081E090E0A0E0B0E08093B8049093B90437
:10291000A093BA04B093BB048091F80384FF1EC057
:102920008091BC049091BD048E7F0E943E0A182FB6
:102930008091B4046091BE040E947F0D082F8091A5
:10294000B504612F0E947F0D282F8091B6046091FD
:10295000B704402F00919B030E9410115D9841988D
:102960008091A7048130D1F0813020F0823009F0CD
:1029700047C034C082E10E94512B892B09F040C02E
:1029800081E08093A7040E941F2A6093A80470939B
:10299000A9048093AA049093AB0432C082E10E9400
:1029A000512B892B21F50E941F2A2091A8043091D8
:1029B000A9044091AA045091AB04621B730B840BD1
:1029C000950B695E734080409040D0F082E0809328
:1029D000A70480ED97E00E94DA1112C082E10E9404
:1029E000512B892B69F080E090E00E94DA1110925F
:1029F000A70406C08091C004883009F058CF55CF95
:102A0000A096EAE00C945B3083E161E00E94B22A78
:102A100083E160E00E941E2B82E08093B00085E09D
:102A20008093B10083E061E00E94B22A83E060E01D
:102A30000E941E2B08951F93182F0E942D2A609329
:102A40009F047093A0048093A1049093A204109318
:102A50008D04112329F440E855E260E070E004C0E1
:102A600040E051EE60E070E089E396E00E943A2E8B
:102A70001F910895ACE1B0E0E0E4F5E10C943F3043
:102A80000E942D2A7B018C0181E00E94A50B54E756
:102A9000A52E6E010894C11CD11C43E0B42EA9825E
:102AA000C60161E00E94CD0FB0929A030E94840C8F
:102AB0006AEF70E080E090E00E94532A80919A03D0
:102AC000833009F07DC089E396E00E94C12E892BF6
:102AD00009F076C00E942D2A6E197F09800B910B98
:102AE0006058734C894C914008F06AC0D8CF8FE78A
:102AF0000E94960A0E94AA0A843509F05CC0898364
:102B00000E94AA0A182F00E010938C0400938B04F3
:102B10000E94AA0A080F111D10938C0400938B04C5
:102B20000E94AA0A80938A040E94AA0A80938904B8
:102B3000813108F040C0FF2407C00E94AA0A07594B
:102B40001B4FF8018083F3940F2D10E080918904CE
:102B500090E0880F991F0817190778F380E7898399
:102B6000CE01019661E00E94CD0F83E080939A032D
:102B70000E94840C62E370E080E090E00E94532A9F
:102B800080919A038330A9F08FE70E94960A0E94F1
:102B9000AA0A803581F4898305EB13E00E94AA0A12
:102BA000F80181938F01F3E0003D1F07B9F781E041
:102BB00003C082E001C083E06C96EAE00C945B30D5
:102BC00080919A03833009F092CFF3CF83E00E9483
:102BD000BA0A8093F90384E00E94BA0A8093FA0348
:102BE00087E061E00E94C00A6AE070E080E090E067
:102BF0000E94532A0E94840C000008950F931F9393
:102C0000082F19C05E9A409A64E670E080E090E078
:102C10000E94532A5E98409864E670E080E090E05D
:102C20000E94532A1F5F101768F36CE271E080E086
:102C300090E00E94532A10E0F6CF482F392F25E06C
:102C40000DC0F999FECF1FBA842F932F92BD81BD7D
:102C500060BD0FB6F894FA9AF99A0FBE215059F058
:102C6000F999FECF842F932F92BD81BDF89A80B53C
:102C7000681739F7089582E00E94FE150895A0E0D4
:102C8000B0E0E5E4F6E10C943830482E562EEE2400
:102C9000FF2488249924C0E0D0E0CC24DD2416E46D
:102CA000312E04C055245394CC24DD24442069F4EF
:102CB00080919B03839DE0011124BCE9EB2EB3E0DE
:102CC000FB2EA9E18A2E912C1DC021E0421671F441
:102CD00080919B03839DE00111246B96F0EDEF2E14
:102CE000F3E0FF2EE9E28E2E912C0CC032E0431669
:102CF00049F47BE9E72E73E0F72E61E0862E912CF4
:102D0000C8E1D1E03E016C0C7D1C1092360510929A
:102D10003505E3011BC0552059F4F999FECFD2BD0A
:102D2000C1BDF89A80B5F701E00FF11F808307C09D
:102D3000F701E00FF11FCE0160810E941D160E0DFC
:102D40001F1DF80180810E94300821969E012619DE
:102D5000022F10E008151905F0F2CE015520D9F424
:102D6000F999FECFD2BDC1BDF89A20B5F999FECF31
:102D70002196D2BDC1BD2197F89A80B590E0B22EC0
:102D8000AA248A299B2920913505309136052817D8
:102D9000390759F487CF2196609136050E941D1698
:102DA000CE01609135050E941D1680E291E0C80EAB
:102DB000D91E91EEC91692E0D90608F477CF852D79
:102DC000CDB7DEB7E1E10C94543080E061E00E94C1
:102DD0003F1681E061E00E943F16089582E061E0C5
:102DE0000E943F16089582E060E00E943F168091A5
:102DF0009B03843020F010929B030E94EE160895EE
:102E00001F93182F0E94F31680919B03811731F0B6
:102E1000143020F410939B030E94EE161F91089526
:102E20001092670485E6E2E0F4E0DF011D928A95E6
:102E3000E9F708951F93182F8F3711F08830E1F5C7
:102E4000E0916704EE2309F455C0E150E093670474
:102E5000F0E0EE5FFB4F108289E396E06DE00E94A8
:102E6000342F10E00AC0E12FF0E0EE5FFB4F89E362
:102E700096E060810E94342F1F5F809167041817CD
:102E800090F389E396E060E20E94342F89E396E0B4
:102E90006DE00E94342F10E00AC0E12FF0E0EE5FF9
:102EA000FB4F89E396E060810E94342F1F5F809181
:102EB0006704181790F31CC08B3119F40E94101787
:102EC0001FC08D30E9F08A30D9F0809167048436D4
:102ED00088F489E396E0612F0E94342F8091670483
:102EE000E82FF0E0EE5FFB4F10838F5F8093670465
:102EF00080E007C089E396E067E00E94E82BF8CF06
:102F000081E01F9108951F93CF93DF93CFEDD3E01E
:102F100010E03BC089E396E062E271E00E94792D07
:102F200089E396E0612F4AE050E00E94F62C89E3A5
:102F300096E06FE271E00E94792D699170E080E087
:102F400090E02091DE0330E040E050E00E94C82F86
:102F500020E137E240E050E00E94C82FDC01CB01C5
:102F60004091D5035091D6036091D7037091D80357
:102F7000480F591F6A1F7B1F89E396E02AE030E063
:102F80000E94BD2C1F5F183119F08881882311F62B
:102F9000DF91CF911F910895EF92FF920F931F93AE
:102FA000882339F489E396E061E77AE00E94062CF1
:102FB0003BC090E00E94B20824E630E040E050E0E0
:102FC0000E94FA2F122F032FF42EE52E622F732F5B
:102FD000842F952F2AE030E040E050E00E94FA2F45
:102FE00089E396E0BA01A9012AE030E00E94AE2C04
:102FF00089E396E06EE20E94E82B612F702F8F2DFF
:103000009E2D2AE030E040E050E00E94FA2FAB0114
:10301000BC0189E396E02AE030E00E94AE2C89E30F
:1030200096E063E70E941A2C1F910F91FF90EF909A
:103030000895FF920F931F93CF93DF9389E396E058
:1030400067E67AE00E94C72B8091B503813041F496
:1030500089E396E06EE47AE00E94062CFF246DC0BE
:10306000823029F489E396E067E37AE0F5CF843093
:1030700029F489E396E063E27AE0EECF853071F7D8
:1030800089E396E068E17AE0E7CFCF2DD0E0C93060
:10309000D1051CF06F2D685C02C06F2D6F5C89E359
:1030A00096E00E94E82B89E396E060E17AE00E94D6
:1030B000C72BBE016F5F7F4F89E396E04AE050E087
:1030C0000E94522D89E396E065E07AE00E94C72BCA
:1030D0008E010B541C4FD8011196EC91E032F8F49C
:1030E00089E396E068EF79E00E94C72BF8018181BF
:1030F000803130F089E396E063E371E00E94792D3E
:10310000CB54DC4F698170E06F7070706F5F7F4FE0
:1031100089E396E04AE050E00E94652D0DC0F0E0A2
:10312000EF70F070EE0FFF1FE75BFC4F6081718165
:1031300089E396E00E947C2DF39480918A04F8162E
:1031400008F4A3CF89E396E06DED79E00E94C72BE8
:103150008091CD030E94CC1789E396E062EC79E080
:103160000E94C72B8091CE030E94CC1789E396E082
:1031700067EA79E00E94C72B8091CF030E94CC17A9
:1031800089E396E06CE879E00E94C72B4091C50383
:103190005091C6036091C7037091C8034115510552
:1031A0006105710539F189E396E02AE030E00E947B
:1031B000BD2C89E396E069E579E00E94C72B8091F8
:1031C000C9030E94E508AB01BC0189E396E02AE04F
:1031D00030E00E94BD2C89E396E065E379E00E942F
:1031E000C72B89E396E06091CA034AE050E00E9451
:1031F000082D06C089E396E06CE279E00E94062C77
:1032000089E396E06FE079E00E94C72B6091CB03E1
:103210007091CC0389E396E04AE050E00E94E22CF2
:1032200089E396E062EF78E00E94C72B6091C403C7
:10323000603450F470E06F5F7F4F89E396E04AE0BE
:1032400050E00E94652D06C089E396E069EE78E0C3
:103250000E94062C89E396E06CEC78E00E94C72B74
:103260008091C30380FD03C065E371E002C069E3A0
:1032700071E089E396E00E947C2D89E396E06FEA95
:1032800078E00E94C72B8091C30382700E94890D51
:1032900089E396E060E978E00E94C72B8091C30340
:1032A00084700E94890D89E396E061E778E00E94CE
:1032B000C72B8091C30388700E94890DCDB7DEB7FC
:1032C000E5E00C9460301F93CF93DF9389E396E0A1
:1032D0006BEB7BE00E94C72B4091D5035091D60346
:1032E0006091D7037091D80389E396E02AE030E03B
:1032F0000E94BD2C89E396E065EA7BE00E94C72B23
:103300004091D9035091DA036091DB037091DC03A3
:1033100089E396E020E130E00E94BD2C89E396E04D
:103320006FE87BE00E94C72B89E396E06091DD03A4
:103330004AE050E00E94082D89E396E069E77BE0CF
:103340000E94C72B89E396E06091DE034AE050E0DB
:103350000E94082D89E396E063E67BE00E94C72B7C
:10336000CFEDD3E010E012C0112331F089E396E0F5
:103370006DE371E00E94792D89E396E069914AE05E
:1033800050E00E94F62C1F5F183119F088818823C5
:1033900059F789E396E00E94F02B89E396E06DE40B
:1033A0007BE00E94C72B89E396E06091F7034AE037
:1033B00050E00E94082D89E396E068E37BE00E94DC
:1033C000C72BE091F803F0E0E770F070EE0FFF1FFD
:1033D000E759FC4F6081718189E396E00E947C2D62
:1033E00089E396E063E27BE00E94C72B8091F803BB
:1033F00090E0887190708830910589F0893091054E
:103400001CF4892B39F01BC08031910569F0489775
:10341000B1F40FC089E396E06AE17BE00EC089E376
:1034200096E06EE07BE009C089E396E068E07BE02F
:1034300004C089E396E06EEF7AE00E94062C89E3EF
:1034400096E06AEE7AE00E94C72B4091D10350913A
:10345000D2036091D3037091D40389E396E02AE00C
:1034600030E00E94BD2C89E396E061ED7AE00E9495
:10347000C72B8091A10380710E94890D89E396E09A
:1034800068EB7AE00E94C72B8091A10380740E94B0
:10349000890D89E396E06FE97AE00E94C72B80915D
:1034A000A10380720E94890D89E396E062E87AE0C8
:1034B0000E94C72B80ED93E00E94F508AB01BC0190
:1034C00089E396E02AE030E00E94AE2C89E396E0A2
:1034D0006DE77AE00E94C72B80ED93E00E94F5082B
:1034E0009B01AC0160E472E48FE090E00E94FA2F4F
:1034F00089E396E0BA01A9012AE030E00E94AE2CEF
:1035000089E396E06AE77AE00E94062CDF91CF918A
:103510001F910895EF92FF920F931F937C0109E38F
:1035200016E0C8016F2D70E04AE050E00E94D12CF7
:10353000C8016EE20E94E82BB70124E076956795FA
:103540002A95E1F76F707070C8014AE050E00E9460
:10355000D12CC8016EE20E94E82B8FE0E822FF2404
:10356000C801B7014AE050E00E94D12C1F910F9191
:10357000FF90EF9008950F931F93CF93DF932091C7
:1035800001042F3FA9F589E396E061EF75E00E9401
:10359000C72B83E793E00E948A1A89E396E060EDE7
:1035A00075E00E94C72B80918B0490918C040E943F
:1035B0008A1A89E396E06DE975E00E94062C89E39A
:1035C00096E06AE775E00E94062C89E396E062E6E1
:1035D00075E00E94062C89E396E06DE375E00E9499
:1035E000062C89E396E00E94F02B0E94191869C00E
:1035F00012160CF066C0332727FD309580918A049F
:1036000090E0821793070CF45CC089E396E068E2CF
:1036100075E00E94C72B60910104772767FD7095C4
:1036200089E396E04AE050E00E94652D89E396E048
:103630006DEF74E00E94C72B08E210E03AC0C12F82
:10364000D0E0CC0FDD1FC759DB4F288130E08091DF
:103650000104992787FD909501972817390741F5AF
:1036600089E396E06FE371E00E94792D89E396E0AB
:10367000602F4AE050E00E94F62C89E396E063E474
:1036800071E00E94792DE981F0E0EF70F070EE0FAB
:10369000FF1FE75BFC4F6081718189E396E00E9428
:1036A000792D89E396E067E471E00E94792D0F5F40
:1036B0001F5F80918904181710F289E396E00E9439
:1036C000F02BDF91CF911F910F910895ACE1B0E005
:1036D000ECE6FBE10C944130282F809101048F3FF0
:1036E00009F042C1822F90E0FC013A97EF36F105D4
:1036F00008F033C1EC5CFF4F0C946E3089E396E028
:1037000069E471E0AEC089E396E069E471E00E948B
:103710007C2D1CC189E396E065E571E00E947C2D5B
:1037200085E78983DE011296E5EBF3E08BE10190FA
:103730000D928150E1F7CE0101966CE10E94CD0F10
:103740000E94840C83E080939A0368EC70E080E030
:1037500090E00E94532A80919A03843009F0FDC0C2
:103760008FE70E94960A0E94AA0A8983853509F08C
:10377000F4C089E396E06FED74E00E94062C89E3C3
:1037800096E061EC74E00E94062C89E396E063EA1F
:1037900074E0ACC089E396E06DE671E00E947C2D98
:1037A00089E68983CE01019661E00E94CD0F0E94D7
:1037B000840C83E080939A0368EC70E080E090E0F2
:1037C0000E94532A80919A03843009F0C6C08FE783
:1037D0000E94960A0E94AA0A89838E010E5F1F4FDB
:1037E000BDE1EB2EF12CEC0EFD1E0E94AA0AD801C1
:1037F0008D938D01AE15BF05C1F7A5EBB3E0FE01BA
:1038000032968BE101900D928150E1F789818934E4
:1038100009F0A3C089E396E065E874E00E94062CF5
:1038200089E396E067E674E00E94062C89E396E05F
:1038300069E474E05BC089E396E067E871E00E94A8
:103840007C2D8EEF8093010488C020522750922F48
:10385000905380918A04891738F489E396E066E9E9
:1038600071E00E947C2D79C0909301046FC084E1C7
:103870008093010489E396E062E174E037C085E15A
:103880008093010489E396E06BED73E02FC086E13D
:103890008093010489E396E064EA73E027C087E13E
:1038A0008093010489E396E06AE573E01FC088E134
:1038B0008093010489E396E069E473E017C089E12D
:1038C0008093010489E396E065E373E00FC08AE129
:1038D0008093010489E396E060E273E007C08BE126
:1038E0008093010489E396E068EF72E00E94062C61
:1038F00034C089E396E06EED72E00E94062C809160
:10390000C30391E01DC089E396E068EC72E00E9479
:10391000062C8091C30392E013C089E396E063EB29
:1039200072E00E94062C8091C30394E009C089E3F1
:1039300096E068E972E00E94062C8091C30398E04B
:1039400089278093C3038FEF809301040E94BB1AE1
:1039500004C089E396E00E94FB2E89E396E00E9472
:10396000C12E892BB1F762C1822F0E941A178823BA
:1039700009F45CC180916704882321F48FEF809360
:1039800001044CC182E094E060E070E040E050E06F
:103990000E94A2069B01AC0160910104862F992729
:1039A00087FD9095A92FB92FFC013197EB31F105D7
:1039B00008F024C1ED55FF4F0C946E30E62FFF2721
:1039C000E7FDF09580918A0490E08E179F070CF434
:1039D00015C1DA01C9010197A109B1098097A105B3
:1039E000B10548F0A8E2FA2E00E010E06F0108945B
:1039F000C108D10825C0EB54FC4F822F8150808331
:103A0000E5C0612F70E0660F771F67597B4FFB01A0
:103A1000808190E08C159D0591F48F2D90E0A0E0C1
:103A2000B0E082179307A407B50741F4F601EB5401
:103A3000FC4FDB0111968C91818301E0F3941F5FB1
:103A4000809189041817E8F2BFC02F3F3105410566
:103A5000510511F008F0D2C02093CD03B7C02F3F1D
:103A600031054105510511F008F0C8C02093CE037F
:103A7000ADC02F3F31054105510511F008F0BEC022
:103A80002093CF03A3C0809102048062803719F590
:103A900083E094E060E070E040E050E00E94A20625
:103AA0009B01AC01DC01CB010197A109B109089789
:103AB000A105B10508F0B5C0CA01B90124ED30E394
:103AC00040E050E00E94C82F9B01AC012A5E3C4AB6
:103AD0004A46554E24C0863611F583E094E060E0F6
:103AE00070E040E050E00E94A2069B01AC01DC01C6
:103AF000CB010197A109B1090797A105B10508F00C
:103B000090C0CA01B90128EA31E640E050E00E94C5
:103B1000C82F9B01AC01245E3C434E46544E2115F8
:103B200031054105510561F0DA01C901805C9D490B
:103B3000A845B54381509A45A246B24008F05EC000
:103B40002093C5033093C6034093C7035093C80323
:103B50003DC02F3F31054105510511F008F04EC021
:103B60002093C90333C0DA01C9010197A109B10942
:103B70008F3F9105A105B10508F040C02093CA030D
:103B800025C0DA01C901845C9940A040B0408D5441
:103B90009D41A040B04030F43093CC032093CB0340
:103BA00001E001C000E0211531054105510511F486
:103BB0008FEF07C0213431054105510528F4822FCC
:103BC00081508093C40302C00023C1F08091680437
:103BD0008823D1F48091D9039091DA03A091DB037B
:103BE000B091DC030196A11DB11D8093D903909380
:103BF000DA03A093DB03B093DC0306C089E396E00D
:103C000068EA71E00E947C2D0E9410178FEF80936C
:103C1000010489E396E06AE00E941A2C0E94BB1A14
:103C200005C021E030E040E050E07ECF6C96E8E057
:103C30000C945D3089E396E06CE472E00E94062CFF
:103C400089E396E064E372E00E94062C89E396E043
:103C50000E94C12E892B31F089E396E00E94FB2E51
:103C60000E94661B0E943A15823019F0833069F475
:103C700005C089E396E066E172E004C089E396E05E
:103C80006FEF71E00E94062C08958FEF809301047E
:103C9000109268040E94BB1A0CC089E396E00E944F
:103CA000C12E892B31F089E396E00E94FB2E0E9401
:103CB000661B809101048E3F81F708958091010475
:103CC000992787FD9095A92FB92FFC013196EB30EC
:103CD000F10508F074C0E254FF4F0C946E3089E394
:103CE00096E064E678E00E94062C83E793E00E9469
:103CF0008A1A89E396E06CE478E00E94062C89E356
:103D000096E067E278E00E94062C89E396E06DEF8A
:103D100077E00E94062C89E396E06CED77E00E9444
:103D2000062C89E396E06FEA77E00E94062C89E38F
:103D300096E069E877E00E94062C89E396E065E664
:103D400077E00E94062C89E396E06EE377E00E941C
:103D5000062C89E396E00E94F02B0E9463192FC085
:103D600089E396E061E277E028C089E396E06CEFB2
:103D700076E023C089E396E067EE76E01EC089E333
:103D800096E068EC76E019C089E396E064E876E0B6
:103D900014C089E396E06FE676E00FC089E396E011
:103DA0006AE576E00E94062C89E396E064E176E01D
:103DB00004C089E396E06EEF75E00E94062C6AE08D
:103DC00070E080E090E00E94532A04C089E396E00E
:103DD0000E94FB2E89E396E00E94C12E892BB1F749
:103DE0000895A2E2B0E0E7EFFEE10C9437308E01D7
:103DF0000F5F1F4F80E1D8011D928A95E9F789E393
:103E000096E066EC71E00E947C2D0E94E61520ECA5
:103E10003DE948E555E32F8F38A349A35AA380EC29
:103E200097EFAAEBB7E38B8F9C8FAD8FBE8F24EFFC
:103E300031E040E050E02F8B388F498F5A8F30E5CA
:103E4000C32E33ECD32EE12CF12C20EC422E2DE9A5
:103E5000522E28E5622E25E3722E882499245401DF
:103E600033241E8A1D8A198A1A8A1B8A1C8AFFC05B
:103E700089E396E00E94FB2E8434B9F0853430F457
:103E80008332B9F18C3209F0CCC044C0833509F0DB
:103E9000C8C02F8D38A149A15AA1C901DA012C014E
:103EA0003D01882499245401E2C089E396E064E44A
:103EB0000E94E82B89E396E040EC5DE968E575E354
:103EC0002AE030E00E941C2D89E396E06CE20E941B
:103ED000E82B89E396E040EC57EF6AEB77E32AE0C2
:103EE00030E00E941C2D89E396E06CE20E941A2CBF
:103EF000BEC019821A821B821C821D821E821F82F2
:103F0000188619861A861B861C861D861E861F86A5
:103F1000188A3AC0339434E0331609F0A8C0698196
:103F20007A818B819C8128EE33E040E050E00E9452
:103F3000C82F6F8F78A389A39AA36D817E818F810B
:103F400098850E94C82F6B8F7C8F8D8F9E8F89855F
:103F50009A85AB85BC858F8B988FA98FBA8F6D851D
:103F60007E858F8598890E94C82F6B017C0190E225
:103F7000C9169EE4D90690E0E90690E0F90630F40F
:103F80008CE162E30E94C00A332471C0A0E3CA1628
:103F9000A5E7DA06A0E0EA06A0E0FA0618F48CE14C
:103FA00062E2F0CFB0E4CB16BCE9DB06B0E0EB0692
:103FB000B0E0FB0618F48CE166E2E4CFE0E5CE1653
:103FC000E3ECDE06E0E0EE06E0E0FE0618F48CE14D
:103FD00062E1D8CFF0E6CF16FAEEDF06F0E0EF06AA
:103FE000F0E0FF0618F48CE165E1CCCF20E7C216C3
:103FF00021E1D20621E0E20620E0F20618F48CE18D
:1040000061E0C0CF30EAC31636E8D30631E0E306FC
:1040100030E0F30618F48CE163E0B4CF8CE165E0A6
:10402000B1CF90ED292E280E49E0421500F1032D65
:1040300010E0000F111F000F111F81E090E08C0FA6
:104040009D1F080F191FD8016D917D918D919C9135
:104050002AE030E040E050E00E94C82F620D711D60
:10406000811D911DF801608371838283938389E3AD
:1040700096E00E94C12E892B09F0FACE811491049A
:10408000A104B10489F4C301B2010E94360B61E0BE
:1040900070E080E090E00E94532AFFEFFE8B1D8AC3
:1040A000198A1A8A1B8A1C8A2F89388D498D5A8D44
:1040B00082169306A406B506E0F40E94E10A298957
:1040C0003A894B895C89280F311D411D511D298B6F
:1040D0003A8B4B8B5C8B3D89381708F48D8B4E895E
:1040E000841708F48E8B0894811C911CA11CB11CB0
:1040F00056C0C301B20128EE33E040E050E00E9418
:10410000FA2F89E396E0BA01A9012AE030E00E9483
:10411000AE2C89E396E06CE20E94E82B89E396E0FE
:104120006D894AE050E00E94F62C89E396E06CE24B
:104130000E94E82B69897A898B899C89A501940161
:104140000E94FA2F89E396E0BA01A9012AE030E043
:104150000E94AE2C89E396E06CE20E94E82B89E392
:1041600096E06E894AE050E00E94F62C89E396E0E2
:104170006CE20E941A2C4C0C5D1C6E1C7F1C8B8DFB
:104180009C8DAD8DBE8D84159505A605B70520F4D3
:104190004F8C58A069A07AA08824992454012F8DAF
:1041A00038A149A15AA1285E33404040504009F04F
:1041B0005ECFA296E2E10C945330A0E0B0E0E3EED3
:1041C000F0E20C9442300E942D2A611571058105A0
:1041D0009105C9F30E9499061092D9031092DA034F
:1041E0001092DB031092DC03DD24E090D903F09001
:1041F000DA030091DB031091DC03102F0F2DFE2C4E
:10420000EE240E9494062FEF30E040E050E00E9440
:104210001C30E60EF71E081F191FE092D903F0921A
:10422000DA030093DB031093DC03D39444E0D41649
:10423000E1F6CFEDD3E000E010E040E1E42E47E20C
:10424000F42E4EC00F5F19F40E944D084DC00E941D
:10425000940622E330E040E050E00E941C306F5FA3
:10426000EFEDF3E090E004C08191861759F39F5F72
:104270009117D0F38091DE0390E08E9D90018F9D89
:10428000300D9E9D300D1124862F90E0AC01249FAF
:10429000C001259F900D349F900D1124AA2797FDF2
:1042A000A095BA2F2091D5033091D6034091D70322
:1042B0005091D803820F931FA41FB51F20919D0317
:1042C00030919E0340919F035091A0032817390716
:1042D0004A075B0708F4B6CF69931F5F183121F0D6
:1042E0008881882309F0AECFCDB7DEB7E7E00C9424
:1042F0005E3080E060E00E943F16882331F081E06C
:1043000060E00E943F16882341F40E9492080E94B8
:104310004D080E94DD200E94E5160895AAE5B0E050
:10432000E4E9F1E20C9443308B017A018B3009F41B
:1043300026C18C3040F5853009F484C0863080F485
:10434000823009F459C0833020F4813009F050C222
:1043500042C0833009F461C0843009F049C265C0AD
:10436000883009F49DC0893038F4863009F486C05D
:10437000873009F03DC28CC0893009F499C08A3079
:1043800009F036C2C9C0893609F482C18A3680F480
:10439000863609F42DC1873620F4853609F028C207
:1043A0000EC1873609F43DC1883609F021C241C1EA
:1043B0008C3609F4C4C18D3638F48A3609F473C1D9
:1043C0008B3609F015C2AFC18D3609F4ECC1873CBC
:1043D00009F00EC200C281E069E270E00E9485111E
:1043E00000ED13E0F80181918F010E946E11F3E05E
:1043F000093F1F07B9F704C282E06BE170E00E9439
:10440000851105EB13E0F80181918F010E946E1177
:10441000F3E0003D1F07B9F7F3C183E061E070E00E
:104420000E9485110E943A15E9C184E061E070E0C4
:104430000E94851181E00E946E110E9467110E9406
:10444000F11EE0C16091890470E0660F771F85E07E
:104450000E94851100E010E008C0F801E759FB4F09
:1044600080810E946E110F5F1F4F8091890490E040
:10447000880F991F0817190780F3C2C186E062E010
:1044800070E00E94851183E793E00E947C11B8C11F
:1044900087E061E070E00E94851180918A04AEC1DE
:1044A00088E061E070E00E94851180919B03A6C1C5
:1044B00086E68983CE01019661E00E94CD0F0E94BD
:1044C000840C83E080939A0368EC70E080E090E0D5
:1044D0000E94532A80919A038430E1F48FE70E946E
:1044E000960A0E94AA0A8983863471F489E060E200
:1044F00070E00E94851110E00E94AA0A0E946E11CD
:104500001F5F1032C9F77CC189E061E070E00E9452
:104510008511C7C089E06DC18AE069E170E00E9441
:10452000851182E080939C038091A305882351F03C
:104530008091A1039091A203A091A303B091A40341
:10454000806809C08091A1039091A203A091A30368
:10455000B091A4038F778093A1039093A203A093BB
:10456000A303B093A4030CE913E0F80181918F0138
:104570000E946E11F3E0053B1F07B9F741C18BE0C4
:1045800061E270E00E9485118091C0048F3F39F094
:104590008091C0048F5F8093C004815002C08091DD
:1045A000C0040E946E1110E0812F0E94A4110E948D
:1045B000190A0E947C111F5F1031B1F721C185E6F5
:1045C00061E070E00E9485110932110509F015C102
:1045D00020E030E0F901E053FC4FD701A20FB31FF8
:1045E0008C9180832F5F3F4F2932310599F759C055
:1045F00086E661E070E00E9485110B31110509F03B
:10460000FCC020E030E0F901EB54FC4FD701A20FD1
:10461000B31F8C9180832F5F3F4F2B31310599F76A
:1046200040C087E661E070E00E9485110E94E516B7
:1046300038C088E661E070E00E94851185E78A83D2
:10464000DE011396E5EBF3E08BE101900D928150D2
:10465000E1F7CE0102966CE10E94CD0F0E94840C1E
:1046600083E080939A0360E273E080E090E00E9430
:10467000532A80919A03843009F0BFC08FE70E94CB
:10468000960A0E94AA0A8A83853509F0B6C009C035
:1046900089E661E070E00E9485110E944D080E9449
:1046A000920881E0ABC08AE661E070E00E9485116B
:1046B00089E68E8FCE014E9661E00E94CD0F0E945A
:1046C000840C83E080939A0360E273E080E090E0E2
:1046D0000E94532A80919A03843009F08EC08FE79C
:1046E0000E94960A0E94AA0A8E8F8E01015E1F4FB9
:1046F0006AE3E62EF12CEC0EFD1E0E94AA0AF801D8
:1047000081938F01EE15FF05C1F7A5EBB3E0FE0124
:104710007F968BE101900D928150E1F78E8D893467
:1047200009F06BC0BECF8BE661E070E00E9485119E
:10473000F70180810E9400170E947921B2CF8CE698
:1047400061E070E00E9485110032110571F487E686
:104750008AAFDE01DB96F70180E201900D92815075
:10476000E1F7CE01CA9661E205C087E48AAFCE01C7
:10477000CA9661E00E94CD0F0E94840C83E0809372
:104780009A036CE474E080E090E00E94532A8091E8
:104790009A03843091F58FE70E94960A0E94AA0A34
:1047A000873459F57ECF8DE661E070E00E94851177
:1047B0000931110511F520E030E0F901E456FC4F14
:1047C000D701A20FB31F8C9180832F5F3F4F2931F8
:1047D000310599F766CF87EC61E070E00E948511A2
:1047E00081E00E946E110E9467111092FF030AC0BF
:1047F0008AEC61E070E00E94851180E00E946E11F9
:104800000E946711C65ADF4FE6E00C945F30A0E0CB
:10481000B0E0EDE0F4E20C943F3084E0A82E06E036
:10482000B02E15E0C12E07E315E0B4E6DB2EA2E0C2
:10483000EA2EF3E0FF2EA1C089E396E00E94FB2E52
:10484000982F8093A2058091A105833021F18430B7
:1048500028F4813099F08230B8F409C0853009F429
:1048600048C0853020F1863009F087C05FC0953B95
:1048700009F083C081E08093A1057FC0923609F0E2
:104880007AC0E092A10579C09093A00590939F050E
:10489000F092A10572C090939D0510929E058091A3
:1048A0009F05892780939F05A092A10566C0D92FF7
:1048B000C0E020919D0530919E052C2B3D2B30931F
:1048C0009E0520939D0580919F05892780939F05D4
:1048D000C092A1052536310508F44FC08CEC61E08B
:1048E00070E00E94851181E00E946E110E946711A4
:1048F00042C020919B0530919C05F901E95CFA4F7B
:10490000908380919F05892780939F052F5F3F4F5C
:1049100030939C0520939B0580919D0590919E0569
:104920002817390750F1B092A10527C080919F0543
:10493000891759F460919B0570919C058091A005A1
:1049400047E355E00E948E210DC08BEC62E070E0E1
:104950000E9485118091A0050E946E118091000433
:104960000E946E11F8018D2D11928A95E9F710922F
:104970009C0510929B051092A10589E396E00E9488
:10498000C12E892B09F058CFCDB7DEB7EAE00C94E1
:104990005B3081E08093FF0308C089E396E00E94CA
:1049A000C12E892B11F00E9407248091FF038823D8
:1049B000A1F708951F93109101041F3F09F0F1C062
:1049C000893409F467C08A3428F5883309F479C03A
:1049D000893368F4803309F486C0813308F06FC0EE
:1049E0008B3109F44DC0813209F0D5C03DC081340E
:1049F00009F49AC0823438F4893309F472C08034DF
:104A000009F0C9C031C0823409F4A1C0863409F06C
:104A1000C2C052C0823609F49AC0833690F48835F9
:104A200079F1893538F4823509F43FC0833509F0CE
:104A3000B2C01FC08A3509F4A9C0813609F0ABC0E5
:104A400073C0823791F1833730F48636A9F1893605
:104A500009F0A1C01FC0883799F08A3709F496C0C1
:104A6000833709F098C005C089E396E069E471E0F6
:104A700019C00E94E51689E396E063ED71E006C077
:104A80000E94792189E396E06DEE71E00E947C2D11
:104A90008EEF7FC00E944D080E94920889E396E045
:104AA0006CE072E00E947C2D76C00E94DD2089E3DC
:104AB00096E065E272E0F6CF0E9483176CC08053E7
:104AC00068C089E396E06CEE71E00E94062C90913C
:104AD000F803892F885F8871977E892B8093F8036C
:104AE00020C089E056C089E396E069ED71E00E943C
:104AF000062C8091A1039091A203A091A303B091F1
:104B0000A40320E130E040E050E082279327A4276F
:104B1000B5278093A1039093A203A093A303B0931E
:104B2000A4031093010437C089E396E063EC71E0BD
:104B30000E94062C8091A1039091A203A091A3034F
:104B4000B091A40320E430E040E050E012C089E3DB
:104B500096E062EB71E00E94062C8091A103909197
:104B6000A203A091A303B091A40320E230E040E0AF
:104B700050E082279327A427B5278093A103909321
:104B8000A203A093A303B093A40302C00E941A1E21
:104B90008FEF80930104809101048E3F09F4DDC002
:104BA000D4C00E941A17882309F4D7C080916704E3
:104BB000882321F48FEF80930104C7C082E094E042
:104BC00060E070E040E050E00E94A2069B01AC0172
:104BD00080910104992787FD9095A92FB92FFC0199
:104BE0003197E930F10508F08CC0E753FF4F0C9482
:104BF0006E30DA01C901815C9D49A845B5438F5FDC
:104C00009945A246B24008F07CC02093D50330936A
:104C1000D6034093D7035093D8039AC02093D90367
:104C20003093DA034093DB035093DC0381E08093FD
:104C300068048EC0283031054105510508F061C077
:104C40002093DD0385C0DA01C9010197A109B109EB
:104C50000A97A105B10508F054C02093DE0378C07F
:104C600082E094E06DE371E00E94BE0710E00EC0A8
:104C7000183130F4E12FF0E0E053FC4F87871F5FDD
:104C800080E090E06DE371E00E94BE07009759F06C
:104C90000E94A007009761F706C0E12FF0E0E05303
:104CA000FC4F17861F5F1831C0F352C02530310505
:104CB0004105510530F52093F7034AC0DA01C901D7
:104CC0000197A109B1090697A105B105D0F480911A
:104CD000F803887F822B8093F8033AC0DA01C90178
:104CE0000197A109B1098050924CA140B04048F40D
:104CF0002093D1033093D2034093D3035093D40332
:104D000027C089E396E068EA71E00E947C2D13C019
:104D10008091D9039091DA03A091DB03B091DC0379
:104D20000196A11DB11D8093D9039093DA03A0933E
:104D3000DB03B093DC030E9410178FEF8093010414
:104D400089E396E06AE00E941A2C0E945E1E05C06C
:104D5000809168048823E1F2EECF1F9108958FEFD0
:104D600080930104109268040E945E1E0CC089E3C7
:104D700096E00E94C12E892B31F089E396E00E94D3
:104D8000FB2E0E94DA24809101048E3F81F76AE0B5
:104D900070E080E090E00E94532A04C089E396E02E
:104DA0000E94FB2E89E396E00E94C12E892BB1F769
:104DB0000895AAE2B0E0EFEDF6E20C943C300E94D8
:104DC0001F2A7B018C0181E00E94A50B04C089E3AE
:104DD00096E00E94FB2E89E396E00E94C12E892B6B
:104DE000B1F75E984098DD24D39432E6732E22E02A
:104DF000822E912C8C0E9D1E5E010894A11CB11C6C
:104E000093E0C92E0E941F2A20E030E06E197F092E
:104E1000800B910B693C71058105910510F021E033
:104E200030E08D2D90E028233923232BA9F10E9417
:104E30001F2A7B018C015D9A419A80ED97E00E94C8
:104E4000DA117982D401E0EDF3E089E201900D926C
:104E50008150E1F7C5016AE20E94CD0F5D9841984B
:104E600080E090E00E94DA11C0929A030E94840CC4
:104E700062E370E080E090E00E94532A80919A0300
:104E8000843051F4C0929A038FE70E94960A0E94E0
:104E9000AA0A823409F4DD2482E10E94512B892B75
:104EA00069F5DD24D3942AC05E9A409A5D9A419AAE
:104EB00089E396E00E94FB2E8D30910569F08E30DB
:104EC00091051CF40A97B1F407C08332910569F08B
:104ED0008234910579F40CC089E396E064EA71E0CC
:104EE0000E94062C0E94AF2605C00E94F11E02C03F
:104EF0000E94C9245E9840985D98419889E396E0A5
:104F00000E94C12E892B09F47DCFCECF8F929F9224
:104F1000AF92BF92CF92DF92EF92FF920F931F93C7
:104F200082E10E94512B892B09F083C068EC70E06C
:104F300080E090E00E94532A80E090E00E94DA1125
:104F40000E941F2A5B016C0140ECE42E42E1F42E2A
:104F5000012D112DE60EF71E081F191F06C082E154
:104F60000E94512B892B09F062C00E941F2A6E15E6
:104F70007F058007910798F382E10E94512B892BCE
:104F800009F055C080ED97E00E94DA110E941F2AB7
:104F90007B018C0199249394882488E496E2A0E014
:104FA000B0E0A80EB91ECA1EDB1E29C0AE14BF0495
:104FB000C006D10638F480ED97E00E94DA1188240B
:104FC00083941DC00E941F2A6E197F09800B910BCC
:104FD000693C71058105910590F00E941F2A7B01B3
:104FE0008C0180E0992009F481E0982E882319F43F
:104FF00080E090E002C080ED97E00E94DA1182E14B
:105000000E94512B892B91F280E090E00E94DA11EE
:10501000882049F080919B038F5F83700E94001766
:105020000E94792106C00E94DD200E94E5160E94A0
:10503000D9261F910F91FF90EF90DF90CF90BF90F6
:10504000AF909F908F90089580E06DEF77E042E001
:1050500050E00E945A290895EF92FF920F931F93F8
:1050600080E00E9419080E94C51186E061E00E945C
:10507000B22A85E061E00E94B22A8EE061E00E94DF
:10508000B22A8FE061E00E94B22A82E160E00E94D1
:10509000B22A88E060E00E94B22A88E061E00E94C3
:1050A0001E2B0E94041589E396E040E052EC61E07B
:1050B00070E00E943A2E0E94F3160E9479210E940D
:1050C000640D8FEF8093C0040E94242878940E947E
:1050D0001F2A7B018C018091C0048F3F09F0DFC043
:1050E0000E941F2A6E197F09800B910B605D77402B
:1050F0008040904008F0D3C0EECF89E396E00E9454
:10510000FB2E89E396E00E94C12E892BB1F789E33B
:1051100096E062E472E00E94792D83E793E00E94BA
:105120008A1A89E396E069E572E00E94792D89E3A5
:1051300096E065E070E04AE050E00E94652D62E391
:1051400070E080E090E00E94532A89E396E00E949C
:10515000C12E04970CF189E396E00E94FB2E823465
:105160009105D1F489E396E00E94FB2E8E349105DF
:1051700099F489E396E00E94FB2E8434910561F452
:1051800089E396E00E94FB2E819731F480E090E065
:105190000E94DA110E94D9264091D1035091D20386
:1051A0006091D3037091D403DB01CA010197A10977
:1051B000B1090497A105B10568F44093C1044330D7
:1051C00029F040E052EC61E070E004C040EA56E8AB
:1051D00061E070E089E396E00E943A2E0E94862703
:1051E0005E98409880E090E00E94DA110E94640D81
:1051F0001092A5048091A10383FF11C08091E50363
:10520000882351F08091EC03882331F08091F303DF
:10521000882311F087E001C085E08093A50480E039
:105220000E94A50B8091A4040E94CB0A0E94840CCA
:1052300010922B0510922C0510922D0510E015C030
:1052400062E370E080E090E00E94532A80ED97E0F6
:105250000E94DA1162E370E080E090E00E94532A3D
:1052600080E090E00E94DA111F5F80919B0381171C
:1052700038F78091F80390E084FF09C020E088713E
:105280009070489709F421E0822F0E941B158FE04F
:105290000E9419081F910F91FF90EF90089580EDE3
:1052A00097E00E94DA1182E161E00E941E2B5E9A73
:1052B000409A27CF823000F5E82FF0E0EE0FFF1F75
:1052C000EC55FA4F71836083882319F08130A1F483
:1052D00008C0809169008C7F842B80936900E89AD4
:1052E000089580916900440F551F440F551F837F17
:1052F000842B80936900E99A08951F920F920FB64C
:105300000F9211242F933F934F935F936F937F934B
:105310008F939F93AF93BF93EF93FF938091A405D7
:105320009091A505892B29F0E091A405F091A505A0
:105330000995FF91EF91BF91AF919F918F917F91CF
:105340006F915F914F913F912F910F900FBE0F90F2
:105350001F9018951F920F920FB60F9211242F9342
:105360003F934F935F936F937F938F939F93AF93ED
:10537000BF93EF93FF938091A6059091A705892B8A
:1053800029F0E091A605F091A7050995FF91EF910D
:10539000BF91AF919F918F917F916F915F914F914D
:1053A0003F912F910F900FBE0F901F9018951F9255
:1053B0000F920FB60F9211242F933F938F939F93C9
:1053C000AF93BF938091AC059091AD05A091AE05D0
:1053D000B091AF053091B0050196A11DB11D232FED
:1053E0002D5F2D3720F02D570196A11DB11D209363
:1053F000B0058093AC059093AD05A093AE05B09336
:10540000AF058091A8059091A905A091AA05B0913A
:10541000AB050196A11DB11D8093A8059093A90528
:10542000A093AA05B093AB05BF91AF919F918F91C7
:105430003F912F910F900FBE0F901F9018958FB72F
:10544000F8942091AC053091AD054091AE05509196
:10545000AF058FBFB901CA0108959FB7F894209195
:10546000A8053091A9054091AA055091AB0586B5D4
:10547000A89B06C08F3F21F02F5F3F4F4F4F5F4FDC
:105480009FBF542F432F322F2227280F311D411D3C
:10549000511D82E0220F331F441F551F8A95D1F7FB
:1054A000B901CA010895EF92FF920F931F93CF9312
:1054B000DF937B018C010E942D2AEB010EC00E941C
:1054C0002D2A6C1B7D0B685E7340C8F30894E108BD
:1054D000F10801091109C851DC4FE114F10401057B
:1054E000110569F7CDB7DEB7E6E00C945F3078942C
:1054F00084B5826084BD84B5816084BD85B58260D9
:1055000085BD85B5816085BDEEE6F0E08081816076
:105510008083E1E8F0E01082808182608083808176
:1055200081608083E0E8F0E0808181608083E1EB4E
:10553000F0E0808184608083E0EBF0E08081816036
:105540008083EAE7F0E080818460808380818260EC
:1055500080838081816080838081806880831092D5
:10556000C1000895CF93DF93482F50E0CA018D5FAB
:10557000934FFC0134914151544FFA018491882397
:1055800069F190E0880F991FFC01EF52F44FA5914B
:10559000B491FC01E552F44FC591D491662351F4C6
:1055A0002FB7F8948C91932F909589238C938881B1
:1055B00089230BC0623061F42FB7F8948C91932F3C
:1055C000909589238C938881832B88832FBF06C075
:1055D0009FB7F8948C91832B8C939FBFDF91CF91D1
:1055E0000895833071F0843028F48130A1F0823046
:1055F00021F514C08630B1F08730D1F08430E9F461
:1056000004C0809180008F7703C0809180008F7DDF
:1056100080938000089584B58F7702C084B58F7D14
:1056200084BD08958091B0008F778093B000089575
:105630008091B0008F7D8093B0000895FF920F930A
:105640001F93F62E482F50E0CA01895E934FFC014C
:105650002491CA018D5F934FFC0114914151544F25
:10566000FA0104910023C9F0222319F0822F0E942D
:10567000F12AE02FF0E0EE0FFF1FE552F44FA59165
:10568000B4919FB7F894FF2021F48C911095812359
:1056900002C08C91812B8C939FBF1F910F91FF9023
:1056A00008950F931F93482F50E0CA01895E934FCE
:1056B000FC012491CA018D5F934FFC01049141517B
:1056C000544FFA011491112319F420E030E015C071
:1056D000222319F0822F0E94F12A812F90E0880F57
:1056E000991F8B51944FFC01A591B4918C9120E0AE
:1056F00030E0802311F021E030E0C9011F910F91CB
:105700000895982F8E3008F09E509770809148032E
:105710008295880F880F807C892B80937C008091F4
:105720007A00806480937A0080917A0086FDFCCFB5
:105730002091780040917900942F80E030E0282B70
:10574000392BC9010895A0E0B0E0E9EAFBE20C942E
:1057500041307C016B018A01C0E0D0E00FC0D6016E
:105760006D916D01D701ED91FC910190F081E02DDB
:10577000C7010995C80FD91F015010400115110527
:1057800071F7CE01CDB7DEB7E8E00C945D30EF9253
:10579000FF920F931F93CF93DF937C018B01C0E0A7
:1057A000D0E0F8010F5F1F4F6491662359F0D701D5
:1057B000ED91FC910190F081E02DC7010995C80F92
:1057C000D91FEFCFCE01CDB7DEB7E6E00C945F3046
:1057D000DC01ED91FC910190F081E02D0995089597
:1057E000EF92FF920F931F938C016DE00E94E82BC4
:1057F0007C01C8016AE00E94E82B9C012E0D3F1D30
:10580000C9011F910F91FF90EF900895EF92FF92C1
:105810000F931F937C010E94C72B8C01C7010E942C
:10582000F02B9C01200F311FC9011F910F91FF9098
:10583000EF900895EF92FF920F931F937C010E94C7
:10584000E82B8C01C7010E94F02B9C01200F311F17
:10585000C9011F910F91FF90EF900895CF93DF93AF
:10586000EC016115710519F420E030E00FC0DB0197
:105870000D900020E9F71197A61BB70BE881F9817D
:105880000280F381E02DAD0109959C01C901DF91F2
:10589000CF9108954F925F927F928F929F92AF9295
:1058A000BF92CF92DF92EF92FF920F931F93DF93FD
:1058B000CF93CDB7DEB7A1970FB6F894DEBF0FBE7A
:1058C000CDBF2C01742ECB01223008F42AE019A29E
:1058D00031E2C32ED12CCC0EDD1E822E9924AA24B7
:1058E000BB24672D752FA50194010E94FA2F790121
:1058F0008A01C801B701A50194010E94C82F472D54
:10590000461B0894C108D1084A3010F4405D01C01C
:10591000495CF6014083E114F1040105110521F011
:105920007E2C5F2DC801DDCFC201B6010E942E2C56
:10593000A1960FB6F894DEBF0FBECDBFCF91DF9119
:105940001F910F91FF90EF90DF90CF90BF90AF909D
:105950009F908F907F905F904F900895DC0121156C
:10596000310541F4ED91FC910190F081E02D642F1F
:10597000099508950E944A2C0895EF92FF920F9383
:105980001F937C010E94AE2C8C01C7010E94F02B5A
:105990009C01200F311FC9011F910F91FF90EF90C3
:1059A0000895EF92FF920F931F939A017B0100E0FD
:1059B00010E0B801A7010E94AE2C1F910F91FF903B
:1059C000EF900895EF92FF920F931F937C010E9436
:1059D000D12C8C01C7010E94F02B9C01200F311F9C
:1059E000C9011F910F91FF90EF900895EF92FF92E0
:1059F0000F931F939A01E62EFF2400E010E0B801F8
:105A0000A7010E94AE2C1F910F91FF90EF90089577
:105A1000EF92FF920F931F937C010E94F62C8C0152
:105A2000C7010E94F02B9C01200F311FC9011F915B
:105A30000F91FF90EF900895A0E0B0E0E2E2FDE268
:105A40000C944130EC016A017B012115310541F4D0
:105A5000E881F9810190F081E02D642F09951BC048
:105A60002A303105B1F477FF13C06DE20E94E82BB4
:105A70008C0144275527BA014C195D096E097F092D
:105A8000CE012AE00E944A2C9C01200F311F04C045
:105A90002AE00E944A2C9C01C901CDB7DEB7E8E09C
:105AA0000C945D30EF92FF920F931F937B019A014C
:105AB0000027F7FC0095102FB801A7010E941C2DAC
:105AC0001F910F91FF90EF900895EF92FF920F9327
:105AD0001F937C010E94522D8C01C7010E94F02B64
:105AE0009C01200F311FC9011F910F91FF90EF9072
:105AF00008950E942E2C0895EF92FF920F931F930A
:105B00007C010E94792D8C01C7010E94F02B9C0121
:105B1000200F311FC9011F910F91FF90EF90089541
:105B200008951F920F920FB60F9211242F933F9357
:105B30004F938F939F93EF93FF938091C00082FDCB
:105B40001DC04091C6002091F1053091F2052F5FF4
:105B50003F4F2F7330708091F3059091F405281713
:105B6000390771F0E091F105F091F205EF54FA4F29
:105B700040833093F2052093F10502C08091C60066
:105B8000FF91EF919F918F914F913F912F910F90A6
:105B90000FBE0F901F9018951F920F920FB60F9285
:105BA00011242F933F938F939F93EF93FF93209113
:105BB00035063091360680913706909138062817C1
:105BC000390731F48091C1008F7D8093C10014C0EA
:105BD000E0913706F0913806EB50FA4F2081809122
:105BE00037069091380601968F739070909338061F
:105BF000809337062093C600FF91EF919F918F917C
:105C00003F912F910F900FBE0F901F901895A0E01D
:105C1000B0E0EDE0FEE20C943D30FC011382128214
:105C200088EE93E0A0E0B0E084839583A683B783F9
:105C30008BE893E0918380837587648757874687D5
:105C4000318B208B138B028BF58AE48AD78AC68A24
:105C5000B18EA08E938E828E8F85848F8889858F5A
:105C60008989868F8A89878F8B8980A32096ECE02B
:105C70000C945930AF92BF92DF92EF92FF920F9344
:105C80001F93CF93DF93EC017A018B01DD24403029
:105C900081EE580780E0680780E0780711F0DD2486
:105CA000D39491E0A92EB12CEC89FD89DD2069F017
:105CB000C50108A002C0880F991F0A94E2F78083EB
:105CC00060E079E08DE390E005C0108260E874E860
:105CD0008EE190E0A80197010E94FA2F21503040F8
:105CE00040405040569547953795279580E12030A4
:105CF000380720F0DD2011F0DD24D6CFE889F989BE
:105D00003083EA89FB89208319A2EE89FF894081CB
:105D100021E030E0C9010C8C02C0880F991F0A9461
:105D2000E2F7482B4083EE89FF894081C9010D8C41
:105D300002C0880F991F0A94E2F7482B4083EE892E
:105D4000FF894081C9010E8C02C0880F991F0A94F7
:105D5000E2F7482B4083EE89FF8980810F8C02C0D7
:105D6000220F331F0A94E2F7209528232083DF9126
:105D7000CF911F910F91FF90EF90DF90BF90AF9068
:105D80000895DC011C96ED91FC911D97E05CFF4F9E
:105D90002191319180819181281B390B2F733070B3
:105DA000C901089589E396E00E94C12E892B11F064
:105DB0000E94902D0895DC011C96ED91FC911D9799
:105DC000E05CFF4F20813181E054F040DF01AE5BA9
:105DD000BF4F8D919C9111972817390719F42FEF18
:105DE0003FEF07C08D919C91E80FF91F8081282F0C
:105DF00030E0C9010895DC011C96ED91FC911D97DE
:105E0000E05CFF4F20813181E054F040DF01AE5B68
:105E1000BF4F8D919C9111972817390719F42FEFD7
:105E20003FEF10C08D919C911197E80FF91F2081D1
:105E30008D919C91119701968F73907011969C9300
:105E40008E9330E0C9010895DC0191968C91919771
:105E5000882339F05496ED91FC915597808186FF07
:105E6000F9CF91961C920895CF93DF93EC01EE85C4
:105E7000FF85E05CFF4F20813181E054F0402F5FCF
:105E80003F4F2F733070DF01AE5BBF4F8D919C9100
:105E9000119728173907D1F3E05CFF4F808191817A
:105EA000E054F040E80FF91F6083EE85FF85E05C69
:105EB000FF4F31832083EE89FF89208181E090E0CC
:105EC0000F8C02C0880F991F0A94E2F7282B2083B9
:105ED00081E089A3EC89FD8980818064808381E0F1
:105EE00090E0DF91CF9108958F929F92AF92BF92F1
:105EF000CF92DF92EF92FF920F931F9300D000D0CA
:105F00000F92EDB7FEB7319684E0ADB7BEB71196EC
:105F10008C9383E0818387E0828385E0838381E0C3
:105F2000848389E396E061EB75E045EF55E025EC6D
:105F300030E004EC10E0B0ECEB2EF12CA1ECCA2E1A
:105F4000D12CF2ECAF2EB12CE6EC8E2E912C0E94CF
:105F5000072E0F900F900F900F900F901F910F91A1
:105F6000FF90EF90DF90CF90BF90AF909F908F9079
:105F70000895CF93DF930E94772A0E942C28C2EDC8
:105F8000DEE20E941C122097E1F30E94D22EF9CF8C
:105F9000629FD001739FF001829FE00DF11D649F0D
:105FA000E00DF11D929FF00D839FF00D749FF00D99
:105FB000659FF00D9927729FB00DE11DF91F639F3A
:105FC000B00DE11DF91FBD01CF011124089597FB0C
:105FD000092E07260AD077FD04D086D006D00020EF
:105FE0001AF4709561957F4F0895F6F79095819515
:105FF0009F4F0895A1E21A2EAA1BBB1BFD010DC0E5
:10600000AA1FBB1FEE1FFF1FA217B307E407F50768
:1060100020F0A21BB30BE40BF50B661F771F881F44
:10602000991F1A9469F760957095809590959B01DA
:10603000AC01BD01CF01089597FB092E05260ED0B6
:1060400057FD04D0D7DF0AD0001C38F45095409596
:10605000309521953F4F4F4F5F4F0895F6F790953C
:106060008095709561957F4F8F4F9F4F08952F9228
:106070003F924F925F926F927F928F929F92AF92D8
:10608000BF92CF92DF92EF92FF920F931F93CF9325
:10609000DF93CDB7DEB7CA1BDB0B0FB6F894DEBFBC
:1060A0000FBECDBF09942A88398848885F846E84E2
:1060B0007D848C849B84AA84B984C884DF80EE802C
:1060C000FD800C811B81AA81B981CE0FD11D0FB635
:1060D000F894DEBF0FBECDBFED010895EE0FFF1F98
:1060E0000590F491E02D0994AA1BBB1B51E107C058
:1060F000AA1FBB1FA617B70710F0A61BB70B881F58
:10610000991F5A95A9F780959095BC01CD010895E6
:10611000911106C0803219F089508550D0F708954A
:0A612000992788270895F894FFCF0F
:10612A004E6F005965730054582074696D656F7518
:10613A007421006D6F64756C65206C6F636B6564A8
:10614A003F00486F70206368616E6E656C200020A6
:10615A0040200053004E2F4100386368002C002C69
:10616A00205B005D20280029004E4F5420454E41F7
:10617A00424C45440053656E64696E6720736574CA
:10618A0074696E677320746F2052580A00526573DF
:10619A00657474696E672073657474696E677320B9
:1061AA006F6E2052580A0041626F727465642065EE
:1061BA00646974730A00696E76616C696420736538
:1061CA006C656374696F6E000D0A496E76616C695D
:1061DA006420696E707574202D206469736361721E
:1061EA006465642107007363616E6E6572206D6F6A
:1061FA0064650053657474696E67732073617665AC
:10620A006420746F20454550524F4D0A00526576FE
:10621A0065727465642073657474696E6773206649
:10622A00726F6D20454550524F4D0A004C6F6164A4
:10623A00656420666163746F72792064656661754E
:10624A006C74730A004B657920616E64206368611F
:10625A006E6E656C732072616E646F6D697A6564C7
:10626A000A004F70656E4C52536E67205458207363
:10627A0074617274696E672000206F6E204857201F
:10628A000050504D00525353490053444100534368
:10629A004C00525844005458440041494E004C4264
:1062AA004545500053504B54524D005342555300EC
:1062BA0053554D44004C4C494E440000342B340095
:1062CA003800382B340031320031322B3400313669
:1062DA000001000000C01200001A400AA1204EA5C9
:1062EA00001B1E27522C23308025000005400AA1DE
:1062FA00204EA50020244EA52C2330004B0000067A
:10630A00400AD0009D49007B289D492C233000E19A
:10631A00000005400A4501D7DC03B81E0EBF002362
:10632A002E48E801008A400A6001555502AD1E2038
:10633A00000023C88025000005400AA1204EA500C0
:10634A0020244EA52C233000020002000200020085
:10635A000200020002000200020002000200020023
:10636A0002000200020002FF01610265026A026E77
:10637A0002720276027A027E0284028B02900295EF
:10638A00029B029B029B029B0235019C02A002A275
:10639A0002A602A902AE02350100070B0C10111564
:1063AA0000160A1322312900000000342FA32BC142
:0863BA002EFB2EDB2E242F0028
:107E00000F92CDB7DEB7112484B714BE81FFF1D035
:107E100082E08093C00088E18093C10086E0809377
:107E2000C20080E18093C4008EE0CDD088249924E4
:107E3000CC24C394F5E0DF2EE1E1EE2E73E0F72EC3
:107E4000B6D0082F813479F4B2D08983C2D0898129
:107E5000823811F481E005C0813811F485E001C059
:107E600083E09ED09AC0823411F484E103C085344B
:107E700019F485E0B6D091C0853561F498D0082F0B
:107E800010E095D090E0982E8824802A912A880CC2
:107E9000991C82C0863521F484E0A3D080E0E1CF34
:107EA000843609F04CC083D082D0A82E80D0B82E62
:107EB00000E011E07CD0F80181938F01AE16D1F77C
:107EC00088D0FB2DF53489F4E0E0F1E00BC0F9999E
:107ED000FECF92BC81BC0894811C911C819180BD15
:107EE000FA9AF99AEA1598F358C08B2D863409F05E
:107EF00054C0F401F7BEE89507B600FCFDCFF401CD
:107F0000A0E0B1E02C9130E011968C91119790E0B7
:107F1000982F8827822B932B12960C01C7BEE895C9
:107F20001124329681E0A038B80761F7F401D7BE7A
:107F3000E89507B600FCFDCFE7BEE8952EC0843774
:107F4000F1F435D034D0182F32D0B82E42D0FB2DDA
:107F5000F63421F4F40105914F010CC0FB2DF534EA
:107F600049F4F999FECF92BC81BC0894811C911C04
:107F7000F89A00B5802F14D0115049F70EC08537FC
:107F800039F427D08EE10CD085E90AD08FE069CF93
:107F9000813511F488E017D01CD080E101D050CF9A
:107FA0009091C00095FFFCCF8093C600089580910A
:107FB000C00087FFFCCF8091C00084FD01C0A89560
:107FC0008091C6000895E0E6F0E098E19083808318
:107FD0000895EDDF803219F088E0F5DFFFCF84E10E
:107FE000DFCF1F93182FE3DF1150E9F7F2DF1F9166
:0E7FF0000895282E80E0E7DFEE27FF27099492
:027FFE0001057B
:0400000300007E007B
:00000001FF
